:1000000012C02AC029C028C027C026C025C024C0CD
:1000100023C022C021C020C01FC01EC01DC01CC0E4
:100020001BC01AC019C011241FBECFEDCDBF10E0F8
:10003000A0E6B0E0EEE4F1E003C0C89531960D9281
:10004000A036B107D1F710E0A0E6B0E001C01D92E4
:10005000A036B107E1F701C0D3CFBF92CF92DF92B4
:10006000EF92FF920F931F93CF93DF938D9ABB9ADA
:1000700083B7816083BF819968C0C39A27E0C22E8D
:10008000D12C9FEFE92E9FEFF92E012D112D82E04B
:10009000B82E80B3682F77276270707012BEC0E0F0
:1000A000D0E040E050E0E0E0F0E082B7242F352FD0
:1000B0002E0F3F1FB32FA22FA80FB11D8A2F9B2FEA
:1000C000AA2797FDA095BA2FE816F9060A071B077D
:1000D00074F188B7882359F4E051FF4F415F5F4FB7
:1000E000C051DF4FB8BE242F352F2C0F3D1F80B3DA
:1000F00099278270907068177907B9F282B7532FE9
:10010000422F480F511D952F842FAA2797FDA095A8
:10011000BA2F8E159F05A007B1074CF482B7280FA0
:10012000311DE22EF32E0027F7FC0095102F0894C6
:10013000C108D108BFEFCB16BFEFDB0609F0A9CF8E
:0E014000819999CF819BFCCF96CFC39894CF25
:00000001FF
